:10000000C828B600841780048413A201201CA20013
:1000100023200319C32823200319C3282320C3281E
:10002000B6005920200821040319C328BD208413D9
:100030003608800664001C281D28A00A0319A10F99
:100040001A288006C3283608A2060130A000A101A4
:10005000000836052206031D0800A00A0319A10F97
:1000600028280800A3003808840036095A20841381
:10007000A3080319C328F030A50022088038A40083
:10008000F030A5030319A5000319A3030319C3281E
:1000900049285D20030120183608A21F3608A2084F
:1000A00003190301A40F562880063D285728000095
:1000B0004028FF3A84178005C3282108200403192B
:1000C000A00A8030201AA1062019A106A018A106B6
:1000D000210DA00DA10DC328A301A200FF30A2078E
:1000E000031CA307031CC3280330A100DF307A20C0
:1000F0006E28A101E83EA000A109FC30031C832862
:10010000A00703188028A0076400A10F80282018EA
:100110008928A01C8D2800008D280800A20001302D
:100120009128A80023082102031D982822082002F4
:10013000043003180130031902302805031DFF3075
:10014000C328A501A4011030A600210DA40DA50D02
:100150002208A4022308031C230FA5020318B728B2
:100160002208A40723080318230FA5070310A00DD6
:10017000A10DA60BA5282008C328A009A109A00A43
:100180000319A10A080083130313831264000800F3
:100190008316023085000130860005308312B800D6
:1001A0000830B6007330A2000A3032203230A2008C
:1001B0000A303220F4204008A0004108A100A30129
:1001C0002F308E20031DDA280530B8000830B60025
:1001D00050304007B20041080318013EB300320816
:1001E000A2000A303220DA280130A000A101053037
:1001F0008400013010200130A0000530840002305E
:1002000001202008BE002108BF003E08A0003F08D2
:10021000A1000F30A200A301A120BC002108BD0055
:100220003E08A0003F08A1000630A200A301A120C3
:10023000C0002108C1000A306C20080063001E299C
:02400E00653F0C
:00000001FF
